S0100000696E706973706D322E73726563E2
S21401F8003F924F925F926F927F928F929F92AF92AA
S21401F810BF92CF92DF92EF92FF920F931F93CF93F7
S21401F820DF93CDB7DEB7A4970FB6F894DEBF0FBE51
S21401F830CDBF89A39AA3CA01F8948095909529A172
S21401F8403AA12817390709F09CC01ABA11BA14BA96
S21401F85017BA1BBA12BA15BA18BADA9AD89AD99A36
S21401F860D29AD09AD19A0E9455FD0E94A7FDD998A6
S21401F870AA24BB2481E090E08BA39CA32501B501BB
S21401F8800E9458FDCE0101960E9443FD382E8D81BF
S21401F890992787FD90958130910539F08230910541
S21401F8A00CF442C00997D9F13FC089819A81E9A138
S21401F8B0FAA18E179F0719F023E0322E35C08E81EC
S21401F8C0EF80F88499E0892E912C8C0E9D1ECC2415
S21401F8D0DD24682E772467FC7094C3010497C8164C
S21401F8E0D90614F587010070A016B10631F0DA9832
S21401F8F0C5010E94D9FC5801DA9AB701C4010E94D9
S21401F9001DFD22E030E0820E931EE20EF31EC20EB3
S21401F910D31EC3010497C816D90624F305C0C50132
S21401F9200E94D9FC82E0382E80E290E0480E591EF3
S21401F9309FEF4916510471F068F00E9455FDEBA146
S21401F940FCA13196EBA3FCA344245524B201CF01BC
S21401F9500E9458FDF1E03F1609F494CF0E9455FD30
S21401F96023E0321611F40E94E8FC81E1F501809350
S21401F9706800E895FFFF0000D99A0E94E8FC81E044
S21401F98090E0A4960FB6F894DEBF0FBECDBFDF9110
S21401F990CF911F910F91FF90EF90DF90CF90BF9086
S21401F9A0AF909F908F907F906F905F904F903F9019
S21401F9B008950F931F938C010E9405FD0E94FCFC85
S21401F9C0C8010E9411FD0E94FCFC1F910F91089531
S21401F9D088E190E029E00FB6F894A89581BD0FBEA6
S21401F9E021BDDA9881E090E00196F1F7DA9A81E09C
S21401F9F090E00196F1F7F5CF80916800089583E1D4
S21401FA000000815087FFFCCF0895FC0183E08093BE
S21401FA106800E895FFFF00008091680080FDFCCF3C
S21401FA200895FC0185E080936800E895FFFF0000DB
S21401FA308091680080FDFCCF0895FC018081918152
S21401FA400C0181E0FB0180936800E895FFFF000050
S21401FA5011248091680080FDFCCF08950F931F93B9
S21401FA6080E00E94B0FD082F112780E00E94B0FDC3
S21401FA70992787FD9095982F8827082B192BC80161
S21401FA801F910F9108951F93CF93DF93EC011FE110
S21401FA9080E00E94B0FD8993115017FFF9CF81E0F5
S21401FAA090E0DF91CF911F910895D39ADB9A089544
S21401FAB0EF92FF921F93CF93DF93CDB7DEB72497D4
S21401FAC00FB6F894DEBF0FBECDBF9C01AB0188E632
S21401FAD08983FE013196C901880F892F881F990BEA
S21401FAE091958F708183220F852F9927280F2B835D
S21401FAF04C83D39ADB987F0113E0F70181917F0154
S21401FB000E94B0FD115017FFF8CF13E08AEA0E9459
S21401FB10B0FD115017FFFACF0E94D2FD80E090E0B1
S21401FB2024960FB6F894DEBF0FBECDBFDF91CF91FE
S21401FB301F91FF90EF90089587E50E94B0FD80E049
S21401FB400E94B0FD8078992787FD90950895959835
S21401FB508D9A939A8B9A92988A9881E090E008956C
S21401FB60282F30E047E027FF02C0939A01C0939800
S21401FB70220F959A330F80B386958695992787FD30
S21401FB80909581709070882311F0316002C000005A
S21401FB9000009598415047FFE6CF832F992787FDB0
S21201FBA090950895959A000000009598089596
S804000000FB
